S3152001700049710120697101200D7001202DE9F0439C
S3152001701006460F464FF0000900253446A84606B11C
S3152001702027B94FF001094846BDE8F08372B600F052
S3152001703095F94FF0000878E040480088B0F5007FC8
S315200170404CD93F48844220D24FF4702000F0BDF83D
S315200170500546002D61D13B48006940F002003949BF
S31520017060086108464461006940F04000086100BF9C
S3152001707000BF4FF4702000F0A8F80546314800699A
S3152001708020F002002F49086147E04FF4702000F0FC
S31520017090C5F80546002D40D12A48006D40F0020072
S315200170A02849086508464465C06900F0020008B110
S315200170B0084644612348006D40F040002149086597
S315200170C000BF00BF4FF4702000F0A8F805461D4808
S315200170D0006D20F002001B4908651EE04FF4702068
S315200170E000F073F80546C5B91648006940F002005C
S315200170F01449086108464461006940F0400008616E
S3152001710000BF00BF4FF4702000F05FF805460D4820
S31520017110006920F002000B49086115B14FF0010901
S3152001712005E004F5006408F10108B84584D300BFE1
S3152001713000F0FEF862B6484676E70000E0F7FF1F4A
S31520017140FFFF07080020024030B50346002441B165
S315200171503AB1002002E01D5C0D54401C9042FAD346
S3152001716000E00124204630BD2DE9F04306460D46B8
S3152001717017464FF00008C14600240EB107B125B9C4
S315200171804FF001084046BDE8F08372B600F0E6F8FC
S3152001719012E015F814306200521CAA5C43EA02215F
S315200171A006EB440000F064F88146B9F1000F02D0E5
S315200171B04FF0010803E0641CB4EB570FE9D300BF7D
S315200171C000F0B6F862B64046DDE700B50346012277
S315200171D000BF00F00BF802465B1E012A01D1002BED
S315200171E0F7D1012A00D10422104600BD00200A4908
S315200171F0C96801F0010109B101200CE00649C968FD
S3152001720001F0100109B1032005E00349C96801F025
S31520017210040101B1022070470020024000B5034657
S31520017220012200BF00F00CF802465B1E012A01D1A3
S31520017230002BF7D1012A00D10422104600BD0000FF
S3152001724000200A49C96C01F0010109B101200CE0B5
S315200172500649C96C01F0100109B1032005E0034973
S31520017260C96C01F0040101B10220704700200240DF
S3152001727070B504460D4600262A480088B0F5007FE1
S3152001728035D92948844219D24FF47020FFF79DFF42
S315200172900646002E43D12548006940F001002349C6
S315200172A0086125804FF47020FFF78FFF06461F489F
S315200172B0006920F001001D49086130E04FF470207B
S315200172C0FFF7ACFF064656BB1848006D40F001009B
S315200172D01649086525804FF47020FFF79FFF064663
S315200172E01248006D20F001001049086517E04FF49F
S315200172F07020FFF76AFF06468EB90C48006940F0F8
S3152001730001000A49086125804FF47020FFF75DFFCF
S3152001731006460648006920F0010004490861304606
S3152001732070BD0000E0F7FF1FFFFF070800200240A5
S315200173300848006940F0800006490861064800882F
S31520017340B0F5007F04D90846006D40F0800008653D
S315200173507047000000200240E0F7FF1F0C4800693B
S3152001736000F0800020B10B48094948600A4848606E
S315200173700A480088B0F5007F09D90548006D00F05C
S31520017380800020B103480249486403484864704795
S315200173900020024023016745AB89EFCDE0F7FF1FAF
S70500000000FA
